:1000000035C04DC04CC04BC04AC049C089C047C074
:1000100046C045C044C043C042C041C040C03FC0CC
:100020003EC03DC03CC0003A370031003B38003292
:1000300000393600300404010104040404040202FF
:100040000202020202020101020201040810204021
:10005000010204081020408004000000000000009D
:1000600002000000010304000000000011241FBE74
:10007000CFEDCDBF10E0A0E6B0E0EAE6F3E002C0CD
:1000800005900D92A036B107D9F710E0A0E6B0E0D8
:1000900001C01D92AD36B107E1F761D164C1B0CFA7
:1000A000EF92FF920F931F9384D07B018C0180E02D
:1000B00021D1019759F4E0926000F0926100009321
:1000C00062001093630084E061E017C080916000DB
:1000D00090916100A0916200B0916300E81AF90A62
:1000E0000A0B1B0B80E4E81687E7F8068BE108078C
:1000F00080E0180718F084E060E0C2D01F910F91F3
:10010000FF90EF90089580E060E07ED080E061E0B5
:10011000B7D084E061E078D084E060E0B1D00895A9
:100120001F920F920FB60F9211242F933F938F932C
:100130009F93AF93BF938091680090916900A091C5
:100140006A00B0916B0030916C00232F2A5F2D372D
:1001500028F02D570396A11DB11D03C00296A11DC5
:10016000B11D20936C008093680090936900A09368
:100170006A00B0936B008091640090916500A0913B
:100180006600B09167000196A11DB11D80936400C7
:1001900090936500A0936600B0936700BF91AF9104
:1001A0009F918F913F912F910F900FBE0F901F90B5
:1001B00018958FB7F89420916800309169004091AC
:1001C0006A0050916B008FBFB901CA0108957894FD
:1001D00080B7836080BF83B7877F83BF83B7887F03
:1001E000836083BF89B7826089BF8EB5887F8EBDEB
:1001F0008FB58C7F81608FBD8EB5877E8EBD8EB5AD
:10020000887F83608EBD0895282F30E0C901895B07
:100210009F4FFC0144912B5C3F4FF901849188234F
:1002200071F1282F30E0F901EA5DFF4FE491AE2F24
:10023000B0E0255D3F4FF9018491E82FF0E066239F
:1002400051F42FB7F8948C91942F909589238C9327
:10025000808189230BC0623061F42FB7F8948C91B0
:10026000942F909589238C938081842B80832FBF3A
:1002700008959FB7F8948C91842B8C939FBF089519
:10028000282F482F50E0CA01895B9F4FFC01349111
:100290004B5C5F4FFA019491992359F12B3019F47B
:1002A00080B78F7304C0273021F480B78F7C80BF64
:1002B0000AC02C3019F48FB58F7304C02D3019F497
:1002C0008FB58F7C8FBDE92FF0E0E55DFF4FE491A6
:1002D000F0E0662341F49FB7F89480813095832342
:1002E00080839FBF08959FB7F8948081832B80837C
:1002F0009FBF0895282F482F50E0CA01895B9F4F68
:10030000FC0194914B5C5F4FFA013491332319F453
:1003100020E030E022C02B3019F480B78F7304C086
:10032000273021F480B78F7C80BF0AC02C3019F4AD
:100330008FB58F7304C02D3019F48FB58F7C8FBDAE
:10034000E32FF0E0E05DFF4FE491F0E0808120E0FA
:1003500030E0892311F021E030E0C901089537DF52
:0A036000D2DE9EDEFECFF894FFCF40
:00000001FF
